:1000000000308A00D128000000000000F7306500B1
:100010000030051901300038031D10281114111685
:10002000F5288E0A3C300E02031C22288E018F0A0E
:100030003C300F02031C22288F01900A1830100256
:1000400003189001FB2814088900831608148312F2
:10005000080895000A301502031C342820301502C8
:1000600003183428063095021A301502031C3A286A
:100070000C30950201301407970017088900831689
:1000800008148312080896000A301602031C4E2832
:100090002030160203184E28063096022030160231
:1000A000031C582830301602031858280C309602CA
:1000B00030301602031C62284030160203186228F2
:1000C0001230960240301602031C6C285030160283
:1000D00003186C281830960250301602031C76283C
:1000E00060301602031876281E309602003411087C
:1000F0004039003803199F28940114088900831699
:100100000814831208088C000C0A03199F28232066
:1001100015081002031D9C2816080F02031D9C28B9
:1001200002301407970017088900831608148312F9
:100130000808FF3A03388600033094077D28FC281E
:100140001730840000080319AD28AB280000000018
:10015000000000000000800BA628B928930A1208AE
:100160001302031DBD28003066000610643097009E
:10017000A0280030660006149301FD2811080139FB
:1001800000380319D0283E30940023201508900031
:1001900016088F008E011117911211100330920072
:1001A000FE288401830104308C008C1DDF28073079
:1001B0008101813084000008C0390F38800064005C
:1001C000813084000008C0390C04800000306600D3
:1001D00006109101013092009301810112309000CC
:1001E0008F018E010B19F6280628F2280B1100301A
:1001F0006600861711287728AE28BE2800306600D2
:060200008613F2286300E2
:02400E00F83F79
:00000001FF
